:10000000A2C00000BCC00000BAC00000B8C0000020
:10001000B6C00000B4C00000B2C00000B0C0000014
:10002000AEC0000066C10000AAC00000A8C6000063
:100030006CC6000013C10000A2C0000016C2000080
:100040009EC000009CC000009AC0000098C0000044
:1000500096C0000094C0000092C000006BC3000076
:100060008EC000008CC000008AC0000088C0000064
:1000700086C0000084C0000082C0000080C0000074
:100080007EC000007CC000007AC0000078C0000084
:1000900076C0000074C000001201100102000008C8
:1000A0004123100001000102DC0109023E000201AF
:1000B00000C0C8090400000102020100052400017B
:1000C0001004240206052406000107058203080027
:1000D000FF09040100020A000000070504024000B5
:1000E00001070583024000010403090432034100B3
:1000F00072006400750069006E006F002000280027
:100100007700770077002E006100720064007500B0
:1001100069006E006F002E0063006300290000007C
:100120002403410072006400750069006E006F00D6
:1001300020004D006500670061002000320035009E
:1001400036003000000011241FBECFEFD4E0DEBF28
:10015000CDBF11E0A0E0B1E0ECE6F4E102C0059013
:100160000D92A037B107D9F712E0A0E7B1E001C0C6
:100170001D92A83DB107E1F73ED30C94340A40CF5D
:100180009C01DC01AE57BF4FED91FC91119741915D
:100190001196FC93EE9380589F4FE817F90711F4DE
:1001A0002D933C939FB7F894F901EC57FF4F808152
:1001B000815080839FBF842F0895429A81E080936D
:1001C0009A0158980895429810929A01589A089561
:1001D000DF93CF930F92CDB7DEB780917201882362
:1001E000F9F48FB78983F89446981092850010929D
:1001F00084008FEF9FEF909389008093880080E4C4
:100200008093800082E08093810080916F00826003
:1002100080936F0081E0809372015D9889818FBF28
:100220000F90CF91DF910895DF93CF930F92CDB7C9
:10023000DEB78FB78983F894EFE6F0E080818D7F99
:1002400080831092800010928100109272015D9A5A
:1002500089818FBF0F90CF91DF9108951F920F92E8
:100260000FB60F9211242F933F934F935F936F9389
:100270007F938F939F93AF93BF93EF93FF9380915F
:100280007201882321F480917301882341F08091C9
:10029000190190911A0190933E0180933D01809144
:1002A0007001823021F480915701882321F08091E0
:1002B0007301882319F08CDF10927301809157012C
:1002C000882309F45C9881E08093570110927101B2
:1002D000FF91EF91BF91AF919F918F917F916F911E
:1002E0005F914F913F912F910F900FBE0F901F90F4
:1002F00018951F920F920FB60F921124EF92FF9252
:100300001F932F933F934F935F936F937F938F939D
:100310009F93AF93BF93CF93DF93EF93FF93C091DE
:100320008400D0918500809170018230C1F4809169
:100330007201882309F078DF189B02C0469A01C039
:10034000469810925701809175018F5F80937501D7
:10035000813808F474C04D9A1092750170C013B1C1
:1003600040917401412751E061E030EEE32E3CEF13
:10037000F32EEC0EFD1E852F842309F43FC0852F3C
:1003800080954823852F8123A62FB0E039F0AA0F4E
:10039000BB1FAA58BE4FCD93DC9330C0FD01EE0FBA
:1003A000FF1FEA58FE4F808191819701281B390B6E
:1003B0008DE02934380738F583E0283E380718F1F6
:1003C000A89510925701FD01E055FE4F80818436BB
:1003D00018F480818F5F8083FD01E256FE4F10820A
:1003E000FD01EE0FFF1FED5CFE4F808191810296B3
:1003F000821B930B059710F031832083442349F02F
:100400006E5F550FB8CF809171018F5F809371013E
:10041000F5CF80917201882309F4DADE80917501AD
:100420008F5F80937501882341F44C9A809171010C
:10043000853618F08FED8093750110937401FF914C
:10044000EF91DF91CF91BF91AF919F918F917F916C
:100450006F915F914F913F912F911F91FF90EF907E
:100460000F900FBE0F901F90189578941F920F92C7
:100470000FB60F9211242F933F938F939F93EF9377
:10048000FF93E0915801F0E0E256FE4F80818932FF
:10049000C0F1809158018830E8F4F89420918800E8
:1004A00030918900E0915801F0E0EE0FFF1FE15F0D
:1004B000FE4F80819181820F931F909389008093DA
:1004C00088007894809158018530C9F481E0809348
:1004D000570115C0F8948091880090918900E091AF
:1004E0005801F0E0EE0FFF1FED5CFE4F20813181DF
:1004F000280F391F309389002093880078945C98E6
:1005000025C0F8942091880030918900E09158012D
:10051000F0E0EE0FFF1FED5CFE4F80819181820FB6
:10052000931F90938900809388007894E0915801FC
:10053000F0E0E055FE4F8081843640F0E0915801B4
:10054000F0E0E256FE4F80818F5F808380915801FA
:100550008F5F8093580180915801823118F010927A
:1005600058014D9AFF91EF919F918F913F912F915B
:100570000F900FBE0F901F90189504B600FC13C08B
:1005800004B601FC10C004B602FE0DC014BE81E02A
:10059000809373018091190190911A0190933E010B
:1005A00080933D0101C014BE3A9A549A559A5C9AC0
:1005B0005D9A80917001882301F522982A9A219AE8
:1005C000299885E3982F9A95F1F793B1969596958A
:1005D00090959170299A8A95F1F71A999F5F2998B9
:1005E00085E38A95F1F71A9905C0923019F4909332
:1005F000700103C081E08093700114B885B18FEF62
:1006000085B9509A80919A01882311F0589801C0B9
:10061000589A80917001823019F481E080936B00C8
:1006200080917001813019F48FEF80936B0080917D
:1006300068008160809368003E9A809170018230EA
:1006400089F088E10FB6F894809360001092600002
:100650000FBEA8958091600088618093600084E45B
:10066000809360000895DF92EF92FF920F931F93A3
:10067000FC018489813019F0823021F405C040E307
:10068000D42E04C0DD2402C030E2D32E8389823010
:1006900011F488E0D82A8589873031F0883031F02C
:1006A000863031F482E003C084E001C086E0D82ABD
:1006B0001092C9001092C8001092CA00E784F08816
:1006C0000189128980E0E81681EEF80680E00807CB
:1006D00080E0180719F420E130E00FC0C801B7012D
:1006E000969587957795679560587B47814E9F4F84
:1006F000A801970197D6215030403093CD00209328
:10070000CC00D092CA0080E0E81681EEF80680E0C6
:10071000080780E0180711F082E001C080E08093B4
:10072000C80088E98093C9001F910F91FF90EF9056
:10073000DF9008951F920F920FB60F9211242F93FE
:100740008F939F93EF93FF939091CE008EB384305D
:10075000F1F4E0914202F09143029083E091420271
:10076000F0914302CF01019690934302809342029D
:100770008254924021F482EC91E0928381839FB76E
:10078000F894809146028F5F809346029FBFFF914D
:10079000EF919F918F912F910F900FBE0F901F900F
:1007A0001895FC01858580FF02C05F9808955F9AC7
:1007B000089589E591E0CCC589E591E07FC587E69C
:1007C00090E09093CD008093CC0086E08093CA00A7
:1007D0001092C80088E18093C900539A5A9A8AB14E
:1007E00080638AB98BB180638BB984D284E085BD84
:1007F0005F9A579A08950F931F93CF93DF93BDDEAF
:10080000DEDF2FB7F89487E492E09093C8028093DC
:10081000C7029093CA028093C9022FBF2FB7F894E2
:1008200082EC91E0909343028093420290934502C0
:10083000809344022FBF7894C7E4D2E003E08FB7DF
:10084000F8949091CB028FBF903809F189E591E03F
:10085000ABD497FD1CC0E091C702F091C802808321
:10086000E091C702F091C802CF0101969093C802AF
:100870008093C702875C924011F4D283C1839FB7F3
:10088000F8948091CB028F5F8093CB029FBF8FB78C
:10089000F894109146028FBFA89902C0113678F1E2
:1008A000A89A80914602882361F05D9800939B018D
:1008B00008C082EC91E064DC682F89E591E0DAD42D
:1008C00011501123B1F780919B01882351F0809141
:1008D0009B01815080939B0180919B01882309F4A7
:1008E0005D9A80919C01882351F080919C018150F8
:1008F00080939C0180919C01882309F45C9A8FB7B6
:10090000F8949091CB028FBF992369F087E492E02D
:1009100037DC982F8091C80085FFFCCF9093CE00E4
:100920005C9800939C0189E591E095D42AD487CF07
:10093000DA01923049F0933061F09130F9F4E8E94E
:10094000F0E022E130E01EC0EAEAF0E02EE330E021
:1009500019C0813049F0813018F0823079F408C034
:10096000E8EEF0E0849107C0ECEEF0E0849103C083
:10097000E0E2F1E08491282F30E004C0E0E0F0E014
:1009800020E030E0ED93FC93C901089528E030E0C9
:1009900040E003C04F5F220F331F28173907D0F301
:1009A000842F8295807F08958093E9008091EB00E9
:1009B00081608093EB001092ED006093EC00409317
:1009C000ED008091EE00881F8827881F08951092FF
:1009D000F40090E09093E9001092F0001092E8008B
:1009E0001092ED008091EB008E7F8093EB009F5F73
:1009F000953081F708958091D00288238CF403C04C
:100A00008EB38823B1F08091E80082FFF9CF809106
:100A1000E8008B778093E80008958EB3882349F02F
:100A20008091E80080FFF9CF8091E8008E77809375
:100A3000E800089594E68091EC0080FF05C0809165
:100A4000E80080FF05C023C08091E80082FD1FC040
:100A50008EB3882311F482E008958EB3853011F4AB
:100A600083E008958091EB0085FF02C081E0089546
:100A70008091E10082FFDFCF8091E1008B7F809346
:100A8000E100992311F484E008959150D4CF80E0DF
:100A900008959C014091D6025091D70246175707FE
:100AA00018F4F90120E038C06115710511F0AB01AF
:100AB000F8CF8091E8008E778093E80040E050E026
:100AC000F0CF8091E80083FF02C081E0089580911B
:100AD000E80082FD2DC08EB3882381F18EB385306E
:100AE00079F18091E80080FF17C09091F20006C074
:100AF00081918093F100415050409F5F4115510515
:100B000011F09830A8F320E0983009F421E08091AA
:100B1000E8008E778093E8004115510591F6222375
:100B200081F606C08EB3882349F08EB3853041F03C
:100B30008091E80082FFF6CF80E0089582E008957A
:100B400083E008959C014091D6025091D702461748
:100B5000570710F490E03BC06115710511F0AB012F
:100B6000F9CF8091E8008E778093E80040E050E074
:100B7000F1CF8091E80083FF02C081E00895809169
:100B8000E80082FD30C08EB3882399F18EB38530A2
:100B900091F18091E80080FF1AC08091F20009C0B5
:100BA000F9012F5F3F4FE491E093F1004150504035
:100BB0008F5F4115510511F0883090F390E0883037
:100BC00009F491E08091E8008E778093E800411568
:100BD000510579F6992369F606C08EB3882349F04A
:100BE0008EB3853041F08091E80082FFF6CF80E03F
:100BF000089582E0089583E008959C0161157105D0
:100C000029F48091E8008B778093E800F90120C0F7
:100C10008091E80083FF02C081E008958EB38823AD
:100C200039F18EB3853031F18091E80082FFF0CF49
:100C300006C08091F10081936150704021F0809155
:100C4000F2008823B1F78091E8008B778093E80069
:100C500061157105E9F606C08EB3882349F08EB39D
:100C6000853041F08091E80080FFF6CF80E0089564
:100C700082E0089583E0089542D044D01EBA1092D5
:100C8000CE021092CD021092CC0284E089BD89B5CB
:100C9000826089BD09B400FEFDCF8091D800982FF5
:100CA0009F779093D80080688093D80080916300EC
:100CB0008E7F809363008091D8008F7D8093D800D1
:100CC0008091E0008E7F8093E0008091E1008E7F34
:100CD0008093E1008091E20081608093E200809146
:100CE000E100877F8093E1008091E200886080933B
:100CF000E2000895C1DF81E08093CF020895109251
:100D0000E20008951092E10008951F920F920FB62D
:100D10000F9211241F932F933F934F935F936F93E1
:100D20007F938F939F93AF93BF93EF93FF93E9EEDE
:100D3000F0E0108117701082E0EFF0E08081877F93
:100D400080837894C3D0F894A9EEB0E01C92E0EFD1
:100D5000F0E08081886080831C93FF91EF91BF91C8
:100D6000AF919F918F917F916F915F914F913F9143
:100D70002F911F910F900FBE0F901F9018951F92EB
:100D80000F920FB60F9211242F933F934F935F93BF
:100D90006F937F938F939F93AF93BF93EF93FF9343
:100DA0008091E10080FF1BC08091E20080FF17C0AE
:100DB0008091E1008E7F8093E1008091E2008E7F40
:100DC0008093E2008091E20080618093E200809154
:100DD000D80080628093D80019BC1EBAF4D98091E3
:100DE000E10084FF29C08091E20084FF25C084E0F7
:100DF00089BD89B5826089BD09B400FEFDCF8091AF
:100E0000D8008F7D8093D8008091E1008F7E809301
:100E1000E1008091E2008F7E8093E2008091E20009
:100E200081608093E2008091CE02882311F481E0FA
:100E300001C084E08EBBC1D98091E10083FF27C04F
:100E40008091E20083FF23C08091E100877F80933F
:100E5000E10082E08EBB1092CE028091E1008E7F95
:100E60008093E1008091E2008E7F8093E200809188
:100E7000E20080618093E200AADD80E060E042E071
:100E800093DD8091F00088608093F00079D18091AB
:100E9000E10082FF0AC08091E20082FF06C08091DB
:100EA000E1008B7F8093E1006BD1FF91EF91BF91C7
:100EB000AF919F918F917F916F915F914F913F91F2
:100EC0002F910F900FBE0F901F9018951F93DF93D7
:100ED000CF93CDB7DEB7AC970FB6F894DEBF0FBE99
:100EE000CDBFE0EDF2E08091F100819322E0E83D9A
:100EF000F207C9F78091D0023091D102353009F460
:100F000087C0363040F43130C9F1313070F03330C1
:100F100009F01DC133C0383009F4EFC0393009F48D
:100F2000FEC0363009F013C192C0803821F08238FB
:100F300009F00DC108C09091CC028091CD028823A8
:100F400099F0926011C08091D40287708093E9007B
:100F50008091EB0090E025E0969587952A95E1F742
:100F6000982F91701092E9008091E800877F80931C
:100F7000E8009093F1001092F100CAC0882319F0A4
:100F8000823009F0E4C090E08F719070009721F0FA
:100F9000029709F0DDC00CC08091D202813009F0C7
:100FA000D7C01092CD02333069F58093CD022AC0AC
:100FB0008091D202882331F52091D402277009F460
:100FC000C7C02093E9008091EB0080FFC1C033309F
:100FD00021F48091EB00806213C08091EB0080616E
:100FE0008093EB0081E090E002C0880F991F2A9562
:100FF000E2F78093EA001092EA008091EB008860AB
:101000008093EB001092E9008091E800877F83C015
:10101000882309F09CC01091D2028091E800877F5C
:101020008093E800E8DC04C08EB3882309F490C004
:101030008091E80080FFF8CF812F8F7711F492E044
:1010400001C093E09EBB80688093E30081C080581C
:10105000823008F07CC08091D2029091D30223E0CC
:101060008C3D920799F55FB7F894DE0115964EE036
:1010700020E030E061E2E42FF0E0609357008491DB
:1010800020FF03C082958F704F5F982F9F70892F2C
:10109000805D8A3308F0895F8C9311961C921197BA
:1010A0002F5F3F4F12962431310529F75FBF8AE247
:1010B0008B8383E08C838091E800877F8093E800B6
:1010C000CE0103966AE270E0E4DC11C06091D402C4
:1010D000AE014F5F5F4F2CDCBC010097C9F18091DE
:1010E000E800877F8093E80089819A812BDD8091D9
:1010F000E8008B778093E8002BC0803841F5809121
:10110000E800877F8093E8008091CE028093F10011
:101110008091E8008E778093E8006DDC19C0882309
:10112000B1F49091D202923098F48091E800877FD8
:101130008093E8009093CE025EDC8091CE028823FB
:1011400011F483E001C084E08EBB36DB01C031DBEB
:101150008091E80083FF0AC08091EB008062809359
:10116000EB008091E800877F8093E800AC960FB693
:10117000F894DEBF0FBECDBFCF91DF911F910895D0
:1011800008951F938EB3882361F01091E9001092A7
:10119000E9008091E80083FF01C098DE177010938A
:1011A000E9001F9108950895FC018EB3843021F564
:1011B00087859089A189B2890097A105B105E1F0E1
:1011C00085818093E9008091E80082FF15C08091BD
:1011D000F200882319F42FEF3FEF04C08091F10053
:1011E000282F30E08091F200882341F48091E800BC
:1011F0008B778093E80002C02FEF3FEFC90108957D
:10120000FC018EB3843011F587859089A189B2895C
:101210000097A105B105D1F081818093E90080910B
:10122000F2008823A9F09091E8008091E8008E7781
:101230008093E80095FD0CC0FDDB982F882349F4CE
:101240008091E8008E778093E80003C092E001C0AF
:1012500090E0892F0895FC018EB3843051F4878586
:101260009089A189B2890097A105B10511F0CF013C
:10127000C7CF08951F93FC01162F8EB38430D9F485
:1012800087859089A189B2890097A105B10599F058
:1012900081818093E9008091E80085FD08C08091FC
:1012A000E8008E778093E800C5DB882329F410934B
:1012B000F10080E001C082E01F9108950F931F9319
:1012C000CF93DF93EC010D96FC0189E0DF011D92C5
:1012D0008A95E9F72A813B8109818C81882311F461
:1012E00010E001C014E0C90151DB182B1260802FFF
:1012F00061E8412F59DB882329F12E813F810D813F
:101300008885882311F410E001C014E0C9013EDB98
:10131000182B1260802F60E8412F46DB882391F064
:101320002A853B8509858C85882311F410E001C04E
:1013300014E0C9012BDB182B1260802F61EC412FC8
:1013400033DB01C080E0DF91CF911F910F910895B1
:10135000CF93DF93EC018091E80083FF60C0888128
:1013600090E02091D4023091D5022817390709F076
:1013700056C08091D102813261F0823220F48032F5
:1013800009F04DC019C0823269F1833209F047C0BB
:1013900038C08091D002813A09F041C08091E800C4
:1013A000877F8093E800CE010F9667E070E071DBE5
:1013B0008091E8008B7713C08091D002813279F55B
:1013C0008091E800877F8093E800CE010F9667E068
:1013D00070E013DCCE0147D98091E8008E778093CE
:1013E000E8001DC08091D0028132C9F48091E800EC
:1013F000877F8093E8008091D2028D87CE01D1D97A
:101400000DC08091D002813251F48091E800877F35
:101410008093E800CE016091D202C5DEECDADF9164
:10142000CF910895A1E21A2EAA1BBB1BFD010DC08E
:10143000AA1FBB1FEE1FFF1FA217B307E407F50784
:1014400020F0A21BB30BE40BF50B661F771F881F60
:10145000991F1A9469F760957095809590959B01F6
:0C146000AC01BD01CF010895F894FFCF4E
:10146C004172647550504D76322E332E3137002038
:10147C00039808200398082003E803200398082009
:10148C0003060920039808200398082003980820D5
:10149C00030852200398082003980820037805209D
:1014AC0003980820030609200398082003980820B5
:1014BC000398082003085201110003400000044067
:1014CC000000020800000000000000000000000006
:00000001FF
